S01E000062696E2F64656D6F70726F675F73746D3332663734362E7372656322
S31508008000000005207D860008CD860008CD8600087C
S31508008010CD860008CD860008CD8600080000000041
S31508008020000000000000000000000000CD860008E7
S31508008030CD86000800000000CD86000805870008E8
S31508008040CD860008CD860008CD860008CD860008B6
S31508008050CD860008CD860008CD860008CD860008A6
S31508008060CD860008CD860008CD860008CD86000896
S31508008070CD860008CD860008CD860008CD86000886
S31508008080CD860008CD860008CD860008CD86000876
S31508008090CD860008CD860008CD860008CD86000866
S315080080A0CD860008CD860008CD860008CD86000856
S315080080B0CD860008CD860008CD860008CD86000846
S315080080C0CD860008CD860008CD860008CD86000836
S315080080D0CD860008CD860008CD860008CD86000826
S315080080E0CD860008CD860008CD860008CD86000816
S315080080F0CD860008CD860008CD860008CD86000806
S31508008100CD860008CD860008CD860008CD860008F5
S31508008110CD860008CD860008CD860008CD860008E5
S31508008120CD860008CD860008CD860008CD860008D5
S31508008130CD860008CD860008CD860008CD860008C5
S31508008140CD860008CD860008CD860008CD860008B5
S31508008150CD860008CD860008CD860008CD860008A5
S31508008160CD860008CD860008CD860008CD86000895
S31508008170CD860008CD860008CD86000800000000E0
S31508008180CD860008CD860008CD860008CD86000875
S31508008190CD860008CD860008CD860008CD86000865
S315080081A0CD860008CD860008CD860008CD86000855
S315080081B0CD860008CD860008CD860008CD86000845
S311080081C0CD860008CD860008EE11AA55F1
S315080081CC10B5054C237833B9044B13B10448AFF3F7
S315080081DC00800123237010BD340400200000000029
S315080081ECC4A00008084B10B51BB108490848AFF3E2
S315080081FC00800848036803B910BD074B002BFBD059
S3150800820CBDE81040184700BF0000000038040020E5
S3150800821CC4A00008340400200000000053B94AB971
S3150800822C002908BF00281CBF4FF0FF314FF0FF3064
S3150800823C00F07EB9ADF1080C6DE904CE00F006F835
S3150800824CDDF804E0DDE9022304B070472DE9F047B8
S3150800825C8C460E460446089D002B50D18A4217467A
S3150800826C6CD9B2FA82FEBEF1000F0BD0CEF1200407
S3150800827C20FA04F401FA0EF644EA060C02FA0EF792
S3150800828C00FA0EF44FEA1749220CBCFBF9F01FFA58
S3150800829C87F809FB10C642EA064600FB08F3B34208
S315080082AC09D9F61900F1FF3280F02281B34240F267
S315080082BC1F8102383E44F61AA2B2B6FBF9F309FB43
S315080082CC136642EA064403FB08F8A04509D9E419E3
S315080082DC03F1FF3280F00A81A04540F20781023B88
S315080082EC3C44C8EB040443EA00400021002D62D04C
S315080082FC24FA0EF400232C606B60BDE8F0878B42E1
S3150800830C07D9002D55D0002185E841000846BDE85F
S3150800831CF087B3FA83F1002940F09080B34202D378
S3150800832C824200F2F880841A66EB03060120B446F2
S3150800833C002D40D085E81010BDE8F08712B901274A
S3150800834CB7FBF2F7B7FA87FEBEF1000F35D1F31B70
S3150800835C4FEA17481FFA87FC0121B3FBF8F0220CE9
S3150800836C08FB103642EA06460CFB00F3B34207D963
S3150800837CF61900F1FF3202D2B34200F2CE80104653
S3150800838CF61AA2B2B6FBF8F308FB136642EA0644E1
S3150800839C0CFB03FCA44507D9E41903F1FF3202D2FE
S315080083ACA44500F2B5801346CCEB040443EA00401E
S315080083BC9CE729462846BDE8F087CEF1200106FA47
S315080083CC0EF307FA0EF720FA01F94FEA1748CE40D2
S315080083DC49EA0309B6FBF8FA4FEA194408FB1A6688
S315080083EC1FFA87FC44EA06430AFB0CF29A4200FA87
S315080083FC0EF40AD9DB190AF1FF3180F087809A420C
S3150800840C40F28480AAF1020A3B449B1A1FFA89F9A6
S3150800841CB3FBF8F108FB113349EA034301FB0CF6ED
S3150800842C9E4207D9DB1901F1FF326BD29E4269D9FC
S3150800843C02393B449B1B41EA0A418EE7C1F1200EE7
S3150800844C22FA0EF48B40234320FA0EF706FA01F4AF
S3150800845C4FEA134C26FA0EF63C43B6FBFCF9270CEE
S3150800846C0CFB19661FFA83F847EA064609FB08F758
S3150800847CB74202FA01F200FA01FA08D9F61809F11C
S3150800848CFF3041D2B7423FD9A9F102091E44F61B67
S3150800849CA0B2B6FBFCF40CFB146640EA064704FBD8
S315080084AC08F8B84507D9FF1804F1FF3028D2B845A3
S315080084BC26D9023C1F4444EA0940C8EB0707A0FB2F
S315080084CC02894F4544464E4614D329D065B3BAEBB8
S315080084DC040367EB060707FA0EFECB40CF404EEABD
S315080084EC030385E888000021BDE8F0871346F8E603
S315080084FC1046E0E6B8EB020469EB03060138E5E73B
S3150800850C0446D8E7114695E78146C0E78A467CE7D4
S3150800851C023B3C4448E708460AE702383E442FE744
S3150800852CC245E7D33E46D1E72946BDE8F08700BFEA
S3150800853C704700BF70B50F4E0F4D761BB61018BF9F
S3150800854C002405D0013455F8043B9847A642F9D1C6
S3150800855C0A4E0B4D761B01F0AFFDB61018BF002462
S3150800856C06D0013455F8043B9847A642F9D170BD9C
S3150800857C70BD00BF24A1000824A100082CA1000886
S3150800858C24A10008024B13B1024800F005B8704745
S3150800859C00000000B1850008002301461A4618465B
S315080085AC00F014B838B5074D074C2C1BA41005D091
S315080085BC013C55F8043D9847002CF9D1BDE83840E4
S315080085CC01F080BD30A100082CA100082DE9F04768
S315080085DC254C2568D5F8484106468846924699465C
S315080085ECC4B360681F2817DC431C76B104EB8005FE
S315080085FC0122C5F888A0D4F8881182401143022EAE
S3150800860CC4F88811C5F808911ED00230636044F886
S3150800861C20800020BDE8F087144B03B34FF4C870D4
S3150800862CAFF300800446D0B1D5F84831002780E86E
S3150800863C8800C5F8484138460123C4F88871C4F83F
S3150800864C8C71002EE1D0D1E7D4F88C110A43C4F80A
S3150800865C8C21DAE705F5A674C5F84841C1E74FF051
S3150800866CFF30BDE8F08700BFDCA000080000000062
S3150800867CDFF834D0002103E00C4B5B58435004312F
S3150800868C0B480C4B42189A42F6D30B4A02E00023CD
S3150800869C42F8043B094B9A42F9D300F023F9FFF749
S315080086AC49FF00F083F870470000052030A1000848
S315080086BC0000002034040020340400203C0500206F
S315080086CCFEE7000008B500F075FF084BA3FB003069
S315080086DC800901F007F9042001F01AF90022114665
S315080086EC4FF0FF3001F0CEF808BD00BFD34D621035
S315080086FC08B501F073FB08BD08B501F063FB01F082
S3150800870C19F908BD00B595B0214B1A6C42F0805288
S3150800871C1A641B6C03F080530193019B1D4B1A685A
S3150800872C42F440421A601B6803F440430293029BCE
S3150800873C012308934FF4A023099302230E934FF4B5
S3150800874C80020F92082210924FF4D872119212934B
S3150800875C139308A800F014FC00B1FEE700F050FFD4
S3150800876C00B1FEE70F23039302230493002305931A
S3150800877C4FF4A05306934FF480530793072103A88D
S3150800878C00F062FE00B1FEE715B05DF804FB00BF11
S3150800879C003802400070004008B501F007FBFFF7EF
S315080087ACB1FFFFF78FFF01F01FFB08BD08B5FFF7F8
S315080087BCF3FF01F0F3FB01F021FB01F077FCFAE77C
S315080087CCF0B58DB0444B1A6C42F080521A641A6C90
S315080087DC02F080520192019A5A6C42F480425A6411
S315080087EC5A6C02F480420292029A1A6B42F0020206
S315080087FC1A631A6B02F002020392039A1A6B42F07E
S3150800880C08021A631A6B02F008020492049A1A6C8C
S3150800881C42F480221A641A6C02F480220592059A94
S3150800882C1A6C42F000721A641B6C03F00073069300
S3150800883C069B032001F014F8002211466FF00B007A
S3150800884C01F020F8002211466FF00A0001F01AF820
S3150800885C002211466FF0090001F014F800221146A7
S3150800886C6FF0040001F00EF8002211466FF00300B9
S3150800887C01F008F8002211466FF0010001F002F829
S3150800888C002211464FF0FF3000F0FCFF80230793BF
S3150800889C01230893002409940A9407A90F4800F0A9
S315080088ACEFFE4FF4407307930227089709940325A4
S315080088BC0A9507230B930A4E07A9304600F0E0FEEB
S315080088CC0795089709940A9509230B9307A9304627
S315080088DC00F0D6FE0DB0F0BD003802400004024090
S315080088EC000C02400C4AD2F8883043F47003C2F8E4
S315080088FC88300A4B1A6842F001021A600021996006
S3150800890C1868074A02401A60064A5A601A6822F41E
S3150800891C80221A60D960704700ED00E000380240EA
S3150800892CFFFFF6FE10300024704700BF2DE9F0411A
S3150800893C05460F4616469846069C1EE0B4F1FF3FC0
S3150800894C1BD02CB101F04AFAC8EB0000844214D8AB
S3150800895C2A68136823F4D07313602A68936823F083
S3150800896C01039360202385F8693085F86A30002363
S3150800897C85F868300320BDE8F0812B68DB6937EA97
S3150800898C03030CBF01230023B342D7D00020BDE854
S3150800899CF08100BF2DE9F04182B01E4690F86A308E
S315080089ACDBB2202B71D104460D469046002A18BF1F
S315080089BC00296CD090F86830012B6AD0012380F816
S315080089CC68300023C366222380F86A3001F006FA61
S315080089DC0746A4F85880A4F85A80A368B3F5805FB4
S315080089EC0AD1236923B940F2FF13A4F85C301AE0C4
S315080089FCFF23A4F85C3016E04BB923691BB9FF2397
S31508008A0CA4F85C300FE07F23A4F85C300BE0B3F1DC
S31508008A1C805F08D123691BB97F23A4F85C3002E078
S31508008A2C3F23A4F85C30B4F85C8022E0B4F85A30E2
S31508008A3C9BB2013B9BB2A4F85A3000963B460022E7
S31508008A4C20212046FFF772FF28BBA368B3F5805F89
S31508008A5C08D1236933B923685B6A08EA030325F846
S31508008A6C023B06E023685B6A5FFA88F213402B70B8
S31508008A7C0135B4F85A309BB2002BD7D1202384F891
S31508008A8C6A30002084F8680006E0022004E0012021
S31508008A9C02E0022000E0032002B0BDE8F08100BF2E
S31508008AAC38B50446826803691A4343691A43C3698D
S31508008ABC1A4301680868A34B034013430B602168EB
S31508008ACC4B6823F44052E36813434B60A269236A4C
S31508008ADC1A4321688B6823F4306313438B6025682B
S31508008AEC994B9D4213D103F59433D3F8903003F088
S31508008AFC0303032B03D8DFE803F0D406040810237A
S31508008B0CE0E00223DEE00423DCE00823DAE08F4B06
S31508008B1C9D4218D103F5FA33D3F8903003F00C03C1
S31508008B2C0C2B08D8DFE803F0BF0707070B07070766
S31508008B3C090707070D001023C4E00223C2E004232B
S31508008B4CC0E00823BEE0824B9D4218D103F5F833EA
S31508008B5CD3F8903003F03003102B0CD003D8002B2D
S31508008B6C00F0A38003E0202B03D0302B05D0102374
S31508008B7CA8E00223A6E00423A4E00823A2E0754B90
S31508008B8C9D4218D103F5F633D3F8903003F0C003A1
S31508008B9C402B0CD003D8002B00F0898003E0802BE7
S31508008BAC03D0C02B05D010238CE002238AE00423C3
S31508008BBC88E0082386E0684B9D421AD103F5F43306
S31508008BCCD3F8903003F44073B3F5807F0DD002D8F8
S31508008BDC002B6ED005E0B3F5007F04D0B3F5407FCB
S31508008BEC05D010236EE002236CE004236AE0082308
S31508008BFC68E05A4B9D421AD103F59233D3F890305C
S31508008C0C03F44063B3F5806F0DD002D8002B52D015
S31508008C1C05E0B3F5006F04D0B3F5406F05D010230B
S31508008C2C50E002234EE004234CE008234AE04C4B68
S31508008C3C9D4219D103F5E033D3F8903003F4405331
S31508008C4CB3F5805F0CD001D8BBB305E0B3F5005F74
S31508008C5C04D0B3F5405F05D0102333E0022331E08E
S31508008C6C04232FE008232DE03E4B9D4227D103F524
S31508008C7CDE33D3F8903003F44043B3F5804F0CD071
S31508008C8C01D8F3B105E0B3F5004F04D0B3F5404F66
S31508008C9C05D0102316E0022314E0042312E008235F
S31508008CAC10E001230EE000230CE000230AE0002369
S31508008CBC08E0002306E0012304E0002302E0102369
S31508008CCC00E00023E269B2F5004F59D1082B4DD8C4
S31508008CDCDFE803F005101B4C244C4C4C2F0000F01D
S31508008CEC6FFC63685A0802EB4000B0FBF3F39BB2C7
S31508008CFC00203DE000F074FC63685A0802EB400063
S31508008D0CB0FBF3F39BB2002032E06268164B03EB20
S31508008D1C5203B3FBF2F39BB2002029E000F02EFBC2
S31508008D2C63685A0802EB4000B0FBF3F39BB20020D1
S31508008D3C1EE06268530803F58033B3FBF2F39BB26B
S31508008D4C002015E0F369FFEF0010014000440040D5
S31508008D5C00480040004C0040005000400014014000
S31508008D6C00780040007C00400048E8010120002300
S31508008D7C23F00F02C3F3420313432268D36038BDB2
S31508008D8C082B3BD8DFE803F005101B3A253A3A3A8C
S31508008D9C300000F015FC636800EB5300B0FBF3F0F1
S31508008DAC80B2E860002038BD00F01AFC636800EB5E
S31508008DBC5300B0FBF3F080B2E860002038BD62685F
S31508008DCC0F4B03EB5203B3FBF2F39BB2EB600020A1
S31508008DDC38BD00F0D3FA636800EB5300B0FBF3F030
S31508008DEC80B2E860002038BD6268530803F500437A
S31508008DFCB3FBF2F39BB2EB60002038BD012038BD03
S31508008E0C0024F400436A13F0010F06D001684B687E
S31508008E1C23F40032836A13434B60436A13F0020F40
S31508008E2C06D001684B6823F48032C36A13434B603F
S31508008E3C436A13F0040F06D001684B6823F48022AA
S31508008E4C036B13434B60436A13F0080F06D0016893
S31508008E5C4B6823F40042436B13434B60436A13F08D
S31508008E6C100F06D001688B6823F48052836B13436A
S31508008E7C8B60436A13F0200F06D001688B6823F4C5
S31508008E8C0052C36B13438B60436A13F0400F11D027
S31508008E9C01684B6823F48012036C13434B60036C14
S31508008EACB3F5801F06D101684B6823F4C002436CE6
S31508008EBC13434B60436A13F0800F06D001684B6866
S31508008ECC23F40022836C13434B60704710B582B0B1
S31508008EDC04460023C36600F081FF2268126812F06C
S31508008EEC080F0AD06FF07E430093034600224FF416
S31508008EFC00112046FFF71AFD40B9202384F8693083
S31508008F0C84F86A30002084F8680000E0032002B078
S31508008F1C10BD00BF80B310B5044690F8693013F045
S31508008F2CFF0F04D1002380F86830FFF7FDFC2423DB
S31508008F3C84F869302268136823F00103136020460D
S31508008F4CFFF7AEFD012819D0636A13B12046FFF767
S31508008F5C59FF2268536823F4904353602268936838
S31508008F6C23F02A0393602268136843F00103136005
S31508008F7C2046FFF7ABFF10BD0120704710BD00BFA0
S31508008F8C002800F0D68170B582B00446036813F049
S31508008F9C010F65D0A64B9B6803F00C03042B0AD073
S31508008FACA34B9B6803F00C03082B0DD1A04B5B68F5
S31508008FBC13F4800F08D09E4B1B6813F4003F4FD058
S31508008FCC6368002B4CD1B6E16368B3F5803F05D1D5
S31508008FDC974A136843F48033136020E04BB9944BDB
S31508008FEC1A6822F480321A601A6822F480221A60EF
S31508008FFC15E0B3F5A02F09D18D4B1A6842F48022DF
S3150800900C1A601A6842F480321A6008E0884B1A68AB
S3150800901C22F480321A601A6822F480221A60636875
S3150800902C7BB100F0DBFE054605E000F0D7FE401BE1
S3150800903C642800F282817E4B1B6813F4003FF4D03F
S3150800904C0EE000F0CBFE054605E000F0C7FE401B1F
S3150800905C642800F27481764B1B6813F4003FF4D134
S3150800906C236813F0020F54D0714B9B6813F00C0F46
S3150800907C0AD06F4B9B6803F00C03082B16D16C4B6C
S3150800908C5B6813F4800F11D1694B1B6813F0020F40
S3150800909C03D0E368012B40F05481654A136823F02A
S315080090ACF803216943EAC103136032E0E368E3B1CC
S315080090BC5F4A136843F00103136000F08FFE054600
S315080090CC05E000F08BFE401B022800F23C81584B51
S315080090DC1B6813F0020FF4D0554A136823F0F803F3
S315080090EC216943EAC103136013E0514A136823F05C
S315080090FC0103136000F072FE054605E000F06EFEF3
S3150800910C401B022800F22181494B1B6813F0020F01
S3150800911CF4D1236813F0080F2AD06369A3B1444A23
S3150800912C536F43F00103536700F058FE054605E0FC
S3150800913C00F054FE401B022800F209813C4B5B6F81
S3150800914C13F0020FF4D013E0394A536F23F00103DE
S3150800915C536700F043FE054605E000F03FFE401B52
S3150800916C022800F2F680324B5B6F13F0020FF4D133
S3150800917C236813F0040F00F083802D4B1B6C13F03F
S3150800918C805F0BD12A4B1A6C42F080521A641B6C06
S3150800919C03F080530193019B012500E00025254B24
S315080091AC1B6813F4807F13D1224A136843F4807327
S315080091BC136000F013FE064605E000F00FFE801B58
S315080091CC642800F2C8801B4B1B6813F4807FF4D00C
S315080091DCA368012B05D1164A136F43F001031367D5
S315080091EC1FE04BB9124B1A6F22F001021A671A6F5D
S315080091FC22F004021A6714E0052B09D10C4B1A6FDE
S3150800920C42F004021A671A6F42F001021A6708E064
S3150800921C074B1A6F22F001021A671A6F22F0040222
S3150800922C1A67A368B3B100F0D9FD06460CE000BF77
S3150800923C003802400070004000F0D0FD801B41F25F
S3150800924C8833984200F289804B4B1B6F13F0020F40
S3150800925CF2D00FE000F0C2FD064606E000F0BEFDB7
S3150800926C801B41F28833984279D8434B1B6F13F015
S3150800927C020FF3D125B1404A136C23F080531364C3
S3150800928CA369002B6DD03C4A926802F00C02082A9E
S3150800929C69D0022B38D1384A136823F080731360CF
S315080092AC00F09CFD054604E000F098FD401B0228E2
S315080092BC5BD8314B1B6813F0007FF5D1E269236A42
S315080092CC1343626A43EA8213A26A5208013A43EAD2
S315080092DC0243E26A43EA026343F00053264A5360A8
S315080092EC136843F08073136000F078FD044604E0BD
S315080092FC00F074FD001B022839D81F4B1B6813F0AD
S3150800930C007FF5D0002035E01B4A136823F08073E4
S3150800931C136000F063FD044604E000F05FFD001BDB
S3150800932C022826D8144B1B6813F0007FF5D10020B1
S3150800933C20E00120704701201CE003201AE00320DE
S3150800934C18E0012016E0032014E0032012E00320A5
S3150800935C10E003200EE003200CE003200AE00320B3
S3150800936C08E0002006E0012004E0032002E00320C8
S3150800937C00E0032002B070BD0038024038B52F4B10
S3150800938C9B6803F00C03042B55D0082B01D02C48F2
S3150800939C38BD2A4B5A6802F03F025B6813F4800FFB
S315080093AC20D0264B5B68C3F38813DC0000256901C3
S315080093BC41EAD4616001041B61EB0505A90141EA88
S315080093CC9461A001001B61EB0501C01841F1000175
S315080093DC4B0243EAD0534402204619460023FEF7B3
S315080093EC1DFF1FE0154B5B68C3F38813DC000025D3
S315080093FC690141EAD4616001041B61EB0505A90109
S3150800940C41EA9461A001001B61EB0501C01841F10A
S3150800941C00018B0243EA9053840220461946002326
S3150800942CFEF7FCFE054B5B68C3F3014301335B0097
S3150800943CB0FBF3F038BD034838BD00BF0038024016
S3150800944C0024F40000127A00002800F09C8070B505
S3150800945C0446544B1B6803F00F038B420BD2514A3C
S3150800946C136823F00F030B431360136803F00F0301
S3150800947C994240F08A80236813F0020F17D013F034
S3150800948C040F04D0484A936843F4E0539360236866
S3150800949C13F0080F04D0444A936843F4604393606E
S315080094AC4148836823F0F002A368134383600D4692
S315080094BC236813F0010F2ED06268012A05D13A4BA6
S315080094CC1B6813F4003F0DD161E0022A05D1364B17
S315080094DC1B6813F0007F05D15BE0334B1B6813F058
S315080094EC020F58D030498B6823F0030313438B6063
S315080094FC00F074FC064606E000F070FC801B41F296
S3150800950C8833984249D8284B9B6803F00C03626849
S3150800951CB3EB820FF0D1234B1B6803F00F039D426C
S3150800952C0AD2204A136823F00F032B4313601368DF
S3150800953C03F00F039D4232D1236813F0040F06D0B3
S3150800954C19498B6823F4E052E36813438B6023684C
S3150800955C13F0080F07D0144A936823F46043216963
S3150800956C43EAC1039360FFF709FF0F4B9B68C3F3EC
S3150800957C03130E4AD35CD8400D4B1860002000F03C
S3150800958CEFFB002070BD01207047012070BD012043
S3150800959C70BD012070BD012070BD032070BD012077
S315080095AC70BD00BF003C024000380240E0A0000835
S315080095BC28040020014B1868704700BF28040020B7
S315080095CC08B5FFF7F7FF044B9B68C3F38223034ADE
S315080095DCD35CD84008BD00BF00380240F0A0000894
S315080095EC08B5FFF7E7FF044B9B68C3F34233034AFE
S315080095FCD35CD84008BD00BF00380240F0A0000874
S3150800960C10B582B01C4B1A6C42F080521A641B6C53
S3150800961C03F080530193019B184A136843F4803373
S3150800962C136000F0DBFB044605E000F0D7FB001BDB
S3150800963CB0F57A7F1AD8114B5B6813F4803FF4D0D7
S3150800964C0E4A136843F40033136000F0C7FB044654
S3150800965C05E000F0C3FB001BB0F57A7F08D8074B72
S3150800966C5B6813F4003FF4D0002002E0032000E00E
S3150800967C032002B010BD00BF003802400070004045
S3150800968CF0B583B00024D8E00123A3400A6803EAA6
S3150800969C0205AB4240F0D0804A68122A18BF022A4B
S315080096AC10D1E608083650F826C004F007029700D1
S315080096BC0F22BA402CEA020E0A69BA404EEA020296
S315080096CC40F82620026867000326BE40F64302EAE5
S315080096DC060E4A6802F00302BA404EEA020202601B
S315080096EC4A6802F1FF3E112A18BFBEF1010F01D9D3
S315080096FC122A10D1826806EA020ECA68BA404EEAE5
S3150800970C02028260426822EA03034A68C2F3001224
S3150800971CA2401A434260C3681E408B68BB40334361
S3150800972CC3604B6813F0805F00F08680454B5A6C1B
S3150800973C42F480425A645B6C03F480430193019BA8
S3150800974CA608B21C404B53F8227004F003039B0086
S3150800975C0F229A4027EA02073C4A904225D002F586
S3150800976C8062904223D002F58062904221D002F5A5
S3150800977C806290421FD002F5806290421DD002F59D
S3150800978C806290421BD002F58062904219D002F595
S3150800979C8062904217D002F58062904215D002F58D
S315080097AC8062904213D1092212E0002210E00122B5
S315080097BC0EE002220CE003220AE0042208E005224D
S315080097CC06E0062204E0072202E0082200E00A224C
S315080097DC02FA03F33B4302361B4A42F826301C4B6B
S315080097EC1A68EB4302EA03064F6817F4803F01D068
S315080097FC45EA0206164A1660526803EA02064F68DC
S3150800980C17F4003F01D045EA0206114A56609268E1
S3150800981C03EA02064F6817F4801F01D045EA0206D0
S3150800982C0B4A9660D26813404E6816F4001F01D096
S3150800983C45EA0203064AD36001340F2C7FF624AF9F
S3150800984C03B0F0BD00380240003801400000024069
S3150800985C003C01400AB18161704709048161704777
S3150800986C064AD36823F4E0631B041B0C000200F4BD
S3150800987CE0601843024B0343D360704700ED00E0E9
S3150800988C0000FA0530B4144BDB68C3F30223C3F1AA
S3150800989C0704042C28BF04241D1D062D01D9DD1E22
S315080098AC00E00025012303FA04F4013C2140A940F9
S315080098BCAB40013B1A400A43002806DA00F00F00B9
S315080098CC1201D2B2054B1A5403E01201D2B2044B60
S315080098DC1A5430BC704700BF00ED00E014ED00E0F0
S315080098EC00E400E00138B0F1807F0AD2064B5860DC
S315080098FCF021064A82F823100020986007221A6085
S3150800990C70470120704700BF10E000E000ED00E052
S3150800991C042805D1054A136843F0040313607047FD
S3150800992C024A136823F004031360704710E000E042
S3150800993C704700BF08B5FFF7FBFF08BD704700BFAF
S3150800994C002800F0A48038B5044690F8203013F0AF
S3150800995CFF0F01D1FFF7F2FF2268136823F0020309
S3150800996C136000F03BFA05460DE000F037FA401B91
S3150800997C0A2808D9636A43F400336362052384F81A
S3150800998C2030012038BD23685A6812F0020FECD13A
S3150800999C1A6842F001021A6000F020FA05460DE03A
S315080099AC00F01CFA401B0A2808D9636A43F40033F2
S315080099BC6362052384F82030012038BD23685A6871
S315080099CC12F0010FECD0227E012A04D11A6842F05B
S315080099DC80021A6003E01A6822F080021A60637E1D
S315080099EC012B05D12268136843F04003136004E089
S315080099FC2268136823F040031360A37E012B05D15C
S31508009A0C2268136843F02003136004E02268136885
S31508009A1C23F020031360E37E012B05D1226813681B
S31508009A2C23F01003136004E02268136843F0100354
S31508009A3C1360237F012B05D12268136843F00803B2
S31508009A4C136004E02268136823F008031360637F2D
S31508009A5C012B05D12268136843F00403136004E054
S31508009A6C2268136823F0040313602168A268E3686C
S31508009A7C1A4323691A4363691A436368013B134300
S31508009A8CCB6100206062012384F8203038BD0120A8
S31508009A9C704700BF70B490F82030DBB2012B05D0AC
S31508009AAC90F82030DBB2022B40F08180434BD3F880
S31508009ABC002242F00102C3F80022D3F8002222F455
S31508009ACC7C52C3F80022D3F80022486A42EA0022E4
S31508009ADCC3F800224A69012000FA02F2D3F81C02E4
S31508009AECD4432040C3F81C02CB69B3B9334BD3F823
S31508009AFC0C022040C3F80C024869CE688D8845EAEA
S31508009B0C0645483043F830504D698E68088840EA57
S31508009B1C0640483503EBC5035860CB69012B16D1B3
S31508009B2C264BD3F80C021043C3F80C0248690E688E
S31508009B3C8D8845EA0645483043F830504D698E689D
S31508009B4C888940EA0640483503EBC50358608B699B
S31508009B5C33B91A48D0F804322340C0F8043205E069
S31508009B6C1648D0F804321343C0F804320B6933B9DB
S31508009B7C1248D0F814321C40C0F8144205E00F48BD
S31508009B8CD0F814321343C0F814320B6A012B05D1E2
S31508009B9C0A49D1F81C321A43C1F81C22074AD2F8D2
S31508009BAC003223F00103C2F80032002004E0436AB5
S31508009BBC43F480234362012070BC70470064004064
S31508009BCC38B590F82030DBB2012B22D1044602239B
S31508009BDC80F820300268136823F00103136000F044
S31508009BECFDF805460DE000F0F9F8401B0A2808D9DF
S31508009BFC636A43F400336362052384F8203001203A
S31508009C0C38BD23685B6813F0010FECD10020606245
S31508009C1C38BD436A43F400234362012038BD00BFB4
S31508009C2C30B490F82040E4B2012C05D090F82040CE
S31508009C3CE4B2022C40F08A8051B90468E46814F046
S31508009C4C030F12D1436A43F400134362012084E0E4
S31508009C5C01290AD10468246914F0030F05D1436A53
S31508009C6C43F400134362012077E0056801F11B04F5
S31508009C7C24012C5904F0040494603CB9056801F1DC
S31508009C8C1B0424012C59640D146006E0056801F1C7
S31508009C9C1B0424012C59E4085460056801F11B04C3
S31508009CAC24012D59C5F34005D560056825446D6812
S31508009CBC05F00F051561056825446D68C5F307257C
S31508009CCC956105682C446468240C546104680A017F
S31508009CDC1444D4F8B8411C7004681444D4F8B84138
S31508009CEC240A5C7004681444D4F8B841240C9C709B
S31508009CFC04681444D4F8B841240EDC70046814447F
S31508009D0CD4F8BC411C7104681444D4F8BC41240A28
S31508009D1C5C7104681444D4F8BC41240C9C71046826
S31508009D2C2244D2F8BC21120EDA7131B90268D36812
S31508009D3C43F02003D36000200FE001290CD1026800
S31508009D4C136943F020031361002006E0436A43F4C9
S31508009D5C80234362012000E0002030BC704700BF1E
S31508009D6C10B504460E4B18784FF47A73B3FBF0F320
S31508009D7C0C4A1068B0FBF3F0FFF7B4FD58B90F2C7A
S31508009D8C0BD8002221464FF0FF30FFF77BFD064B20
S31508009D9C1C60002010BD012010BD012010BD00BFA5
S31508009DAC30040020280400202C04002008B50320C9
S31508009DBCFFF756FD0020FFF7D3FFFEF701FD002045
S31508009DCC08BD00BF034A1368034909780B4413609E
S31508009DDC704700BF3805002030040020014B186876
S31508009DEC704700BF3805002008B5002280210248BC
S31508009DFCFFF730FD08BD00BF0004024010B5FEF7A2
S31508009E0C77FC0E4B1B68C31AB3F5FA7F14D30446BA
S31508009E1C0B4B1B783BB90122094B1A708021094858
S31508009E2CFFF718FD06E00022054B1A70802105483D
S31508009E3CFFF710FD014B1C6010BD00BF500400203D
S31508009E4C540400200004024008B50948094B036075
S31508009E5C4FF46143436000238360C36003610C22A3
S31508009E6C42618361C36103624362FFF753F808BD1D
S31508009E7C58040020004800402DE9F04104460D46E0
S31508009E8C17469846FFF79CFB154BA3FB0030800939
S31508009E9C00221FE0134B13F8121003EB420393F83E
S31508009EAC01E001EB0E0303FB0443B0FBF3FC03FBDD
S31508009EBC1C066EB91FFA8CF32B80013B9BB2B3F5CB
S31508009ECC806F05D2397088F800E00120BDE8F08172
S31508009EDC0132D2B2112ADDD90020BDE8F08100BFCB
S31508009EECD34D6210F8A0000830B58DB00025ADF83A
S31508009EFC2E508DF82D500CAB03F8045D0DF12D0288
S31508009F0C0DF12E014FF4FA70FFF7B6FF1A4C1B4BE6
S31508009F1C236025766576A576E57625776577A5603B
S31508009F2CE5609DF82D30013B1B0423619DF82C3010
S31508009F3C013B1B056361BDF82E3063602046FFF7B5
S31508009F4CFFFC06950795012308934CF6E04201920F
S31508009F5C02954FF6E0720392042204920595099332
S31508009F6C0E230A930DEB02012046FFF793FD2046BC
S31508009F7CFFF726FE0DB030BD0C050020006400402E
S31508009F8C08B50023012201460348FEF703FD08B96C
S31508009F9C012008BD002008BD5804002008B5FFF7AD
S31508009FAC53FFFFF7A1FF08BDBFF34F8F0549CA68DA
S31508009FBC02F4E062044B1343CB60BFF34F8F00BF30
S31508009FCCFDE700BF00ED00E00400FA0508B5214BDB
S31508009FDC1B78ABB92048FFF7D3FF012838D11E4BA5
S31508009FEC1B78013BDBB23F2B32D8FEF781FB1B4BB0
S31508009FFC18600122174B1A700022194B1A7008BDEB
S3150800A00C174B1B78013314481844FFF7B9FF01287E
S3150800A01C14D1134A13780133DBB213700E4A127833
S3150800A02C934215D100220B4B1A700B4B5B78FF2B06
S3150800A03C0ED1094B9B785BB9FFF7B6FFFEF758FBB9
S3150800A04C064B1B686433984202D90022014B1A70DE
S3150800A05C08BD00BF0A050020C804002034050020EE
S3150800A06C0905002000B58BB001AB03AA00210E48E8
S3150800A07CFFF7D6FDA8B940F26763039A9A4203D153
S3150800A08C059B1BB1002302E0002300E0012343B12A
S3150800A09C9DF80430FF2B04D19DF805300BB9FFF75A
S3150800A0AC83FF0BB05DF804FB0C05002008B5FFF721
S3150800A0BC8DFFFFF7D7FF08BDF8B500BFF8BC08BC85
S3150800A0CC9E467047F8B500BFF8BC08BC9E4670475C
S3150800A0DC000000200000000000000000010203043C
S3150800A0EC060708090000000001020304050206021F
S3150800A0FC060307030803090309040A040B040C04E2
S3150800A10C0C050D050E050F050F0610061007100891
S30D0800A11C3CE1FF7F0100000091
S30D0800A12491850008F18100088D
S3090800A12CCD810008CB
S3150800A13000000000EC02002054030020BC030020AD
S3150800A1400000000000000000000000000000000001
S3150800A15000000000000000000000000000000000F1
S3150800A16000000000000000000000000000000000E1
S3150800A17000000000000000000000000000000000D1
S3150800A18000000000000000000000000000000000C1
S3150800A19000000000000000000000000000000000B1
S3150800A1A000000000000000000000000000000000A1
S3150800A1B00000000000000000000000000000000091
S3150800A1C00000000000000000000000000000000081
S3150800A1D00000000000000000010000000000000070
S3150800A1E00E33CDAB34126DE6ECDE05000B00000035
S3150800A1F00000000000000000000000000000000051
S3150800A2000000000000000000000000000000000040
S3150800A2100000000000000000000000000000000030
S3150800A2200000000000000000000000000000000020
S3150800A55000000000000000000024F40010000000C5
S3090800A56001000000E8
S7050800867DEF
